:10000000C2C000000C94BB1B0C94E21B0C94091C96
:100010000C94301C0C943C14E5C00000E3C00000BC
:10002000E1C00000DFC000000C942F2B0C94AC2B1F
:10003000D9C00000D7C00000D5C000000C94B11397
:10004000D1C000000C948213CDC00000CBC00000D2
:100050000C944D13C7C00000C5C000000C94C82A02
:10006000C1C00000BFC00000BDC00000BBC0000098
:10007000B9C00000B7C00000B5C00000B3C00000A8
:100080000C94551B0C942114ADC00000ABC00000B3
:10009000A9C00000A7C000008B15D91502163016A4
:1000A0005C1665167316CD164B179617A517E31732
:1000B000F2176F1886180001000067011200020095
:1000C0000024014300030000200104010309040689
:1000D000011802030904EE001603030904E0000CF2
:1000E0000C033100320033003400350000001603E9
:1000F0005500530042002000530065007200690063
:1001000061006C00000018035400650065006E007B
:10011000730079006400750069006E006F000000D4
:100120000403090409024300020100C0320904006B
:100130000001020201000524001001052401000154
:100140000424020605240600010705820308004076
:1001500009040100020A0000000705030240000034
:10016000070584024000001201000202000020C0C6
:100170001683040001010203010001C1020180365F
:1001800001813600B11F11241FBECFEFD0E2DEBFC8
:10019000CDBF11E0A0E0B1E0ECE2FEE500E00BBF76
:1001A00002C007900D92A636B107D9F72DE1A6E659
:1001B000B1E001C01D92AF30B207E1F711E0C6E82F
:1001C000D1E000E006C022970109FE010BBF0E94AA
:1001D0006D2EC438D10780E00807A9F70E94552A80
:1001E0000C94142F0DCFCF93DF93EC011A8A80E08B
:1001F00090E02FEFFE01E80FF91F20830196803178
:100200009105C1F780E090E021E0FE01E80FF91FC1
:10021000138A178A238F019684309105B1F718A2AB
:100220001F8EFE01E959FF4F108280E189A318A6B5
:100230001FA21AA619A61CA61BA61AA2CE018D964D
:100240000E94F420CE01805C9F4F0E94F420CE01DA
:100250008D5A9F4F0E94F4201BA21CA21DA21EA219
:10026000DF91CF910895CF93DF93EC010E94062197
:10027000CE018D960E940621CE01805C9F4F0E9488
:100280000621CE018D5A9F4F0E940621CE01DF919B
:10029000CF91A9CFFC01128A80E090E02FEFDF011F
:1002A000A80FB91F2C93019680319105C1F780E00A
:1002B00090E021E0DF01A80FB91F53961C925397DD
:1002C00057961C9257975B962C9301968430910514
:1002D00089F712A210A2178E14A613A6CF018D5A69
:1002E0009F4F0C94F420FC01928981A1981768F526
:1002F00082898F5F828B2289222369F0822F90E08E
:10030000DC011197AE0FBF1F3C91DF01A80FB91F91
:100310003C932150F1CF6083278D30A181E090E0A4
:1003200002C0880F991F6A95E2F7822B932B90A346
:10033000878FDF01AA59BF4F8C91882331F0878DB9
:1003400090A19093111C8093101C0895FC0181E0F2
:1003500090E0062E02C0880F991F0A94E2F780955C
:10036000909540E02289DF01421708F5A40FB11DE6
:100370002C9126131AC0542F2289521768F4252F66
:1003800030E0D9011196AE0FBF1F7C91DF01A20FA3
:10039000B31F7C935F5FF0CF22892150228B278D82
:1003A00030A12823392330A3278F4F5FDBCFAA59F1
:1003B000BF4F8C91882331F0878D90A19093111CB1
:1003C0008093101C0895FC0122A1211101C0BECF11
:1003D0000895DF92EF92FF920F931F93CF93DF93D5
:1003E000EC01F12CE12C8A89F816B0F48E010F0D86
:1003F000111DF801D080CE010E9461218D1538F4C5
:10040000F801D080CE010E945121D81610F0F3944B
:10041000EACFF801E080FBCF8E2DDF91CF911F91C5
:100420000F91FF90EF90DF900895860F911DFC01D2
:1004300083890895EF92FF920F93CF93DF93EC019E
:10044000E62E642F822FF12C0230A1F00330C9F187
:10045000013009F04BC030E02F5F3F4F442737FD9C
:100460004095542F70E080E090E00E943A2ACE0D33
:10047000DF1D25C09EA1992339F0FE01EE0DFF1D61
:10048000938D913089F544C0CE0DDF1D9B89921369
:1004900002C09FEF9B8F9B89961302C091E09B8FB8
:1004A0002B8D9B89332727FD3095290F311D2B8BF1
:1004B0009B89961778F19B89891760F12FC06B8B08
:1004C0002DC0FE01EE0DFF1D9FEF938F93894FEF1F
:1004D000490F438B691708F0238B9389891708F418
:1004E000838B9EA19923D1F0838B18C0FE01EE0D62
:1004F000FF1D91E0938F93899F5F938B291708F4D9
:10050000438B8389861708F4638B8EA1882331F08F
:10051000638B04C09B8D191694F28B8BDF91CF9166
:100520000F91FF90EF9008953F924F925F926F92DC
:100530007F928F929F92AF92BF92CF92DF92EF9273
:10054000FF920F931F93CF93DF9300D000D0CDB7CE
:10055000DEB79C838B83DC0152968C91529781117C
:1005600009C0453009F455C1042F2FE040E0CD010A
:1005700061DF4FC1433009F4B8C028F4413051F075
:100580004230F9F046C1443009F4E0C0453009F486
:1005900010C13FC1062F10E0EB81FC81228930E0C1
:1005A00040E050E060E070E0CB010E943A2AEB812D
:1005B000FC81E60FF11D8081EB81FC81E00FF11FD2
:1005C00020C1AB81BC8152968C91529770E08230F1
:1005D00008F46CC080E1D82EAD01460F571FFA0118
:1005E0007396FA83E98321E030E0455E5F4FCC24C7
:1005F000C3948A0133243A94AB81BC815F96ED9019
:10060000FC909097A981BA818C91590102C0AA0CE3
:10061000BB1C8A95E2F7C50101978E219F21892B8A
:1006200011F4DA01CC92AB81BC815F96ED90FC9025
:10063000909780818F5F590102C0AA0CBB1C8A95DC
:10064000E2F7C50101972C01662457FC6094762CD3
:10065000409450944701A12CB12C482059206A2085
:100660007B2045284628472811F4D8013C92D80120
:100670008C91F080992787FD90958F0D911D808337
:10068000AB81BC815F96ED90FC9090978081590181
:1006900002C0AA0CBB1C8A95E2F7C5018E219F21DE
:1006A000892B59F4DA9409F0A7CF07C0AB81BC813C
:1006B0008C91FD01E60FF71F838BEB81FC8186A1F6
:1006C000882309F4A6C08F01060F171FD8015B9677
:1006D0008C91813011F4CF0168C08B819C810E9484
:1006E0005121D80153968C9394C00B811C81060F25
:1006F000111D8FEFF801838F60E1739621E030E0E8
:1007000080818150808380818F708083AB81BC81A8
:100710005F964D915C9190978081590102C0AA0C1F
:10072000BB1C8A95E2F7C50184239523892B11F41C
:10073000615031F7AB81BC8196968C919697882356
:1007400009F467C0CD010E94512131C00B811C8189
:10075000060F111D81E0D8015B968C9360E1F801D2
:10076000739621E030E080818F5F808380818F707D
:100770008083AB81BC815F964D915C919097808125
:10078000590102C0AA0CBB1C8A95E2F7C50184235B
:100790009523892B11F4615031F7AB81BC8196967A
:1007A0008C9196978823A9F1CD010E946121F801CF
:1007B00028C0EB81FC81E60FF11D8789882319F1A0
:1007C0009789AB81BC8152968C919817E0F4878908
:1007D0008150878B8789AB81BC81A80FB11D8C911B
:1007E000838BAB81BC8196968C919697882389F0F8
:1007F00052968C9152978150878B8789A80FB11D93
:100800008C91838B06C0AB81BC8152968C91878B77
:10081000DECF0F900F900F900F90DF91CF911F912F
:100820000F91FF90EF90DF90CF90BF90AF909F908F
:100830008F907F906F905F904F903F900895EF92D0
:10084000FF920F931F93CF93DF931F92CDB7DEB725
:100850007C01062F142FDC0152968C91813039F1E6
:1008600038F0823009F443C0833009F467C0A9C06E
:100870002FE040E0612FC701DDDD80E090E09701CF
:10088000210F311DB9016D5E7F4F255E3F4F181757
:1008900049F0FB014081F701E80FF91F438BD901B3
:1008A0004C91438F01968430910589F78AC0C70126
:1008B00040FD05C00E945121282F40E005C00E9444
:1008C000512141E0480F2FE0612FC701B3DD82E0E5
:1008D0008127D701A10FB11D53969C915397F70122
:1008E000E80FF11D938B5B968C91838F6AC0C701D3
:1008F0000E945121282FC70129830E94612129814B
:10090000482F612FC70196DD80E090E09701210F0D
:10091000311DB9016D5E7F4F255E3F4F181749F0BD
:10092000FB014081F701E80FF91F438BD9014C917E
:10093000438F01968430910589F743C0413069F0B7
:1009400028F04230B1F0433059F13BC0C7010E945A
:100950006121282F40E060E032C0C7013ADD282F36
:10096000C70129830E94612141E0480F298161E08C
:1009700026C0C7010E9451218F3058F4C7010E9440
:100980005121282FC701298324DD41E0480F298107
:1009900005C0C7011EDD41E0480F2EE062E00FC038
:1009A000C7010E9451218F3038F4C7010E945121A4
:1009B00041E0480F2FE002C02FE04FE063E0C701A5
:1009C00039DDF70186A1811116A20F90DF91CF9139
:1009D0001F910F91FF90EF900895EF92FF920F9368
:1009E0001F93CF93DF931F92CDB7DEB77C01162FF5
:1009F000FC01E959FF4F8081813009F084C0F70183
:100A00008289813059F030F0823019F1833009F455
:100A10003CC07DC0062F2FE040E026C0C7010E94E9
:100A20005121012F282F40E060E0C70103DDC701FD
:100A30000E94512141E0480F2FE061E0C701FADC3C
:100A4000F7018389858B8489868B838D858F848D3F
:100A50001AC0C7010E945121282FC70129830E9473
:100A60006121012F2981482F60E0C701E3DCF701F4
:100A70008389848B8389858B8389868B838D848FFF
:100A8000838D858F838D868F42C0C7010E9461212F
:100A9000012F282F40E060E0C701CCDCC70199DCC2
:100AA000282FC70129830E94612141E0480F298135
:100AB00061E0C701BFDCC7010E9451218F30A0F463
:100AC000C7010E945121282FC701298382DC41E000
:100AD000480F298162E0C701ADDCC7010E945121A6
:100AE00041E0480F2FE00BC0C70173DC41E0480F25
:100AF000012F2EE062E0C7019DDC2FE04FE063E0B4
:100B0000C70198DC04C0462F60E0C7010DDDF70186
:100B100086A1811116A20F90DF91CF911F910F91A5
:100B2000FF90EF900895FC01E959FF4F108220E1FA
:100B3000FC0121A30895FC01E959FF4F6083613056
:100B400011F423E001C020E1FC0121A30895AF923C
:100B5000BF92CF92DF92EF92FF920F931F93CF93AA
:100B6000DF93EC018AA1882309F445C08E0109595D
:100B70001F4FF80180819E0143E1849F200D311DAC
:100B80001124C9018D960E944321B82E93E1A92E0C
:100B9000EE24E394F12CBB2069F185ED9BE10E94EA
:100BA000E01F6C01BA94F80180819E01A89E200D7F
:100BB000311D1124C9016B2D8D960E944921F70129
:100BC00002C0EE0FFF1F8A95E2F7CF018C219D2115
:100BD000892B09F7F80180819E01A89E200D311D07
:100BE0001124C9016B2D8D960E944921682FCE01D9
:100BF000ADDBD1CF1AA2CA59DF4F8881882321F0FB
:100C00001092111C1092101CDF91CF911F910F9127
:100C1000FF90EF90DF90CF90BF90AF9008950F932B
:100C20001F93CF93DF93EC018C0109591F4FF801FB
:100C300080819E0143E1849F200D311D1124C90153
:100C40008D960E94F420F8018081FE01E80FF11DCD
:100C5000E80FF11D10A617A2DF91CF911F910F9100
:100C60000895CF92DF92EF92FF920F931F93CF934D
:100C7000DF93EC018AA18823B1F0FE01EA59FF4F0E
:100C80008081882309F480C0FE01E959FF4F8081EB
:100C9000C80FD11DC80FD11D8FA198A59093111C0D
:100CA0008093101C71C081E08AA38A898823B9F1DE
:100CB000CE01B5DFDA888E0109591F4F53E1C52EE9
:100CC000EE24E394F12CDD20C1F2DA946D2DCE01F7
:100CD0000E944921F80190819E01C99E200D311D7D
:100CE0001124682FC9018D960E9407216D2DCE0118
:100CF0000E944921F8019081FE01E90FF11DE90FE1
:100D0000F11D27A130A5A70102C0440F551F8A95E8
:100D1000E2F7CA01822B932B90A787A3D4CF8E0131
:100D200009591F4FF801808143E1F42E9E01F89E7E
:100D3000200D311D1124C9018D960E944321882365
:100D400009F49BCFF80180819E01F89E200D311D92
:100D50001124C9018D960E944321F82E33E1E32E20
:100D6000FF2009F48ACFFA94F80180819E01E89E61
:100D7000200D311D1124C9016F2D8D960E9449212E
:100D8000682FCE01B0DAECCFDF91CF911F910F9198
:100D9000FF90EF90DF90CF900895611101C0D7CE02
:100DA00060CFFC01E959FF4F2081FC01E20FF11DEA
:100DB000E20FF11D87A190A521E030E002C0220FD3
:100DC000331F6A95E2F72823392381E0232B09F4A6
:100DD00080E00895BF92CF92DF92EF92FF920F933F
:100DE0001F93CF93DF93EC01D62E8AA181110BC004
:100DF000CE01DF91CF911F910F91FF90EF90DF9087
:100E0000CF90BF9070CACE01CCDF8E0109591F4F21
:100E1000F801811171C08081F3E1FF2E9E01F89EDF
:100E2000200D311D1124C9016D2D8D960E940721C1
:100E3000F80180819E01F89E200D311D1124C90109
:100E40008D960E94432199A1981708F051C0B9A02E
:100E500073E1C72EEE24E394F12CF80180819E010A
:100E6000C89E200D311D1124C9018D960E94432179
:100E7000F8019081B81688F5AE01C99E400D511D4C
:100E80001124CA016B2D8D960E944921682FCE0135
:100E90005DDAF80180819E01C89E200D311D11246C
:100EA000C9016B2D8D960E944921F8019081FE01A8
:100EB000E90FF11DE90FF11D27A130A5A70102C01F
:100EC000440F551F8A95E2F7CA01809590958223B9
:100ED000932390A787A3B394C0CF69A19E0143E158
:100EE000949F200D311D1124C9018D960E94462129
:100EF0006D2DCE01F8D90FC080819E0143E1849F02
:100F0000200D311D1124C9016D2D8D960E942121C6
:100F10006D2DCE011BDAF8018081FE01E80FF11D75
:100F2000E80FF11D27A130A581E090E002C0880FF5
:100F3000991FDA94E2F78227932790A787A3CA59CB
:100F4000DF4F8881882331F087A190A59093111CF1
:100F50008093101CDF91CF911F910F91FF90EF9024
:100F6000DF90CF90BF9008950895CF92DF92FF92C7
:100F70000F931F93CF93DF931F92CDB7DEB78C01F2
:100F8000442381F0FC01128AF62E6B018C2D8F19FF
:100F9000841740F4F60161916F01C80149831ADF9B
:100FA0004981F4CF0F90DF91CF911F910F91FF9066
:100FB000DF90CF900895AF92BF92CF92DF92EF92E1
:100FC000FF920F931F93CF93DF936C018C01035D0E
:100FD0001F4FC8010E944321A82E811114C0A09266
:100FE000321CF60181A592A59093341C8093331C8A
:100FF000DF91CF911F910F91FF90EF90DF90CF90F5
:10100000BF90AF900895BB24BA94B80EC0E0D0E072
:10101000EFEFBE1621F3C0FD0DC06B2DC8010E947D
:1010200049218F70FE01F595E795E65DF34E9081BD
:10103000907F11C07E0181E0E81AF108F594E794F1
:101040006B2DC8010E944921F701E65DF34E8295A0
:10105000807F90819F70982B90832196BA94D8CFEF
:10106000EF92FF920F931F93CF93DF93EC01F090D9
:10107000321CB9D8F11018C08091331C9091341CE7
:10108000892B09F44DC081E0FE01E959FF4F8083AF
:1010900083E089A3CE015BDDCE01E3DD00E010E05B
:1010A000EE24E394F12C29C0FE01E959FF4F108290
:1010B00080E189A3CE014BDDCE01D3DD00E010E05D
:1010C0000F15D0F6F80100FD06C0F595E795E65D31
:1010D000F34E608107C03197F595E795E65DF34ED5
:1010E000608162956F70CE0175DE0F5F1F4FE8CF94
:1010F0000F5F1F4F0031110599F02091331C309183
:10110000341CC701002E02C0880F991F0A94E2F711
:1011100082239323892B61F3602FCE015BDEE8CF1E
:10112000DF91CF911F910F91FF90EF900895FC01F7
:10113000E959FF4F3081FC0122A1E30FF11D23A3E8
:101140000895FC01E959FF4F2081FC01E20FF11DD8
:1011500083A1089521E0FC0126A308958A599F4F99
:1011600021E0FC01208308958A599F4FFC011082E1
:1011700008951092800010928100109282001092C7
:1011800085001092840010926F0010920F1C109234
:101190000E1CAC0120E030E0FC01E20FF31F1082D6
:1011A000FA01F85F118210822F5F3F4F4E5F5F4F51
:1011B000211568E0360781F7FC01F85E1182108284
:1011C00032961182108234961082ED5BFF4F1082AE
:1011D000319623E02083E354F10928E02083089529
:1011E000DC01A75FB74E20E4EBE0F1E001900D9247
:1011F0002A95E1F7BECF6F927F928F929F92AF9226
:10120000BF92CF92DF92EF92FF920F931F93CF93F3
:10121000DF931F92CDB7DEB73C017C0137EBE31AB9
:1012200037EEF30AD7018C91833009F0CFC08301E8
:101230000E5F174EF301EC5FF74E6F01D801ED9191
:10124000FC91E60DF71D608165FD04C08BED9BE10F
:101250000E943013F80180819181FC01FC5FEE0F48
:10126000FF1FE60DF71D20813181232B71F40196BC
:10127000D80111969C938E93F601208131818217BB
:101280009307E1F61D921C92D9CF10928100109223
:101290006F005301F9EFAF1AF7EEBF0AD5018C9139
:1012A000883089F4D801ED91FC91FC5FEE0FFF1FAF
:1012B000E60DF71D808191819093890080938800CD
:1012C00082E080936F00F5018081893044F1430111
:1012D000F4E08F02800C911C112437EF831A37EE53
:1012E000930AD801ED91FC91FC5FEE0FFF1FE60D14
:1012F000F71D6081718180E090E00E94502DF40123
:1013000020813181428153810E94B62D0E94242D7B
:10131000709389006093880082E080936F00D5010C
:101320002C912830E4F5D801ED91FC91FC5FEE0F93
:10133000FF1FE60DF71D6081718180E090E0298339
:101340000E94502D2981F301B4E02B02E00DF11D24
:101350001124E75FF74E20813181428153810E9441
:10136000B62D0E94242DF301E85FF74E8083709321
:101370008900609388008091880090918900892B72
:1013800031F481E090E0909389008093880080811F
:10139000882311F081E001C082E080936F001092F9
:1013A0008500109284008FEF86BB85E080938100DA
:1013B000F80180819181019691838083D6012D91DE
:1013C0003C918217930711F411821082F7018081FA
:1013D000843009F0DDC083010E5F174EDD24D39405
:1013E0007301FCEFEF1AF7EEFF0AD801ED91FC91C3
:1013F000E60DF71D608165FD0AC064FB882780F952
:101400008D2580FB64F98BED9BE10E943013F80180
:1014100080819181FC01FC5FEE0FFF1FE60DF71D3F
:1014200020813181232B81F4892B31F4D7018D91D7
:101430009C91F80191838083D8018D919C911197A3
:1014400001978D939C93D1CF892B41F4F301EC5FED
:10145000F74E80819181F80191838083D8018D912D
:101460009C91119701978D939C93109281001092FB
:101470006F007301B9EFEB1AB7EEFB0AF701808139
:10148000883089F4D801ED91FC91FC5FEE0FFF1FCD
:10149000E60DF71D808191819093890080938800EB
:1014A00082E080936F00F7018081893044F163010D
:1014B000F4E08F02C00CD11C112437EFC31A37EEB1
:1014C000D30AD801ED91FC91FC5FEE0FFF1FE60DF2
:1014D000F71D6081718180E090E00E94502DF6013F
:1014E00020813181428153810E94B62D0E94242D9A
:1014F000709389006093880082E080936F00D70129
:101500002C912830E4F5D801ED91FC91FC5FEE0FB1
:10151000FF1FE60DF71D6081718180E090E0298357
:101520000E94502D2981F301B4E02B02E00DF11D42
:101530001124E75FF74E20813181428153810E945F
:10154000B62D0E94242DF301E85FF74E808370933F
:101550008900609388008091880090918900892B90
:1015600031F481E090E0909389008093880080813D
:10157000882311F081E001C082E080936F00109217
:101580008500109284008FEF86BB85E080938100F8
:101590000F90DF91CF911F910F91FF90EF90DF900F
:1015A000CF90BF90AF909F908F907F906F90089555
:1015B000CF93DF932091840030918500243F41E058
:1015C000340710F425E030E0DC01A75BB74E4C9106
:1015D000423091F4EC01D85EE881F981E150FC4F92
:1015E000EE0FFF1FE80FF91F318320831982188245
:1015F000FC01EE5FF74E13C0443099F4FC01EE5F3E
:10160000F74E208131812F5F3F4F31832083EC01E2
:10161000CC5FD74E488159812417350711F41182C8
:10162000108223E02C93FC01E65BF74E208310929E
:101630000F1C10920E1CDF91CF91DDCDCF93DF9365
:10164000FC01E95FF74E28E02083DC01AC5FB74E78
:101650002D913C911197232BB1F41092850010929B
:10166000840021E020936F003197208325E02093B0
:10167000810022E0ED5BFF4F208320E030E23093D9
:101680000F1C20930E1C4091840050918500443F14
:1016900021E0520710F445E050E010926F001092E4
:1016A00085001092840016BA21E020936F00EC01AF
:1016B000D85E288139816F7D6F7B6F77FC01E20FE7
:1016C000F31F60832115310549F0F901E150FC4F0A
:1016D000EE0FFF1FE80FF91F518340834D915C917E
:1016E00011974F5F5F4F4D935C932F3F374009F445
:1016F0005FDF88819981019699838883DF91CF91FB
:101700000895FC01EC5FF74E208131812F5F3F4F40
:1017100031832083DC01B85EED91FC911197E80FD5
:10172000F91F2081206220832D913C911197211572
:10173000310559F0F901E150FC4FEE0FFF1FE80FA2
:10174000F91F4FEF5FEF518340832F5F3F4F2D9382
:101750003C932115384009F42BCF0895CF93DF93A4
:101760002091840030918500243F41E0340710F43B
:1017700025E030E0DC01A75BB74E4C914230B9F474
:10178000EC01D85EE881F981E150FC4FEE0FFF1FBC
:10179000E80FF91F3183208319821882FC01EC5F66
:1017A000F74E2081318121503109329714C04330E6
:1017B000A1F4FC01EE5FF74E20813181232B39F437
:1017C000EC01CC5FD74E2881398131832083208181
:1017D0003181215031093183208324E02C93FC0195
:1017E000E65BF74E208310920F1C10920E1CDF91C7
:1017F000CF9101CD10920F1C10920E1C10926F0011
:10180000109281001092850010928400FC01F85E15
:1018100011821082E75BFF4F25E020830895CF936C
:10182000DF93EC01E7DF8BED9BE10AD78CE19BE1D5
:1018300097D5C75BD74E1882DF91CF910895FC01F1
:10184000E65BF74E2081233019F0243011F0089523
:10185000AFCE84CFCF93DF93EC018CE19BE180D5B9
:10186000FE01EA5FF74E8081882321F0CE01DF91EF
:10187000CF91E5CFFE01E75BF74E81E08083E55431
:10188000F1091182108280E090EA90930F1C8093FE
:101890000E1C349711821082329611821082C85F1A
:1018A000D74E1882DF91CF910895CF93DF93EC014B
:1018B000FC01E75BF74E80818330C1F050F4823049
:1018C00089F5CE0156DCCE01C5DFDF91CF910C94B6
:1018D00087148430B1F0853029F5FE01E65BF74EC0
:1018E0008081833019F0843061F01CC0CE0197DF15
:1018F000FE01EE5FF74E11821082CE01DF91CF9193
:1019000057CECE018CDFFE01EE5FF74EDE01AC5FFD
:10191000B74E8D919C91019791838083CE01DF9189
:10192000CF911CCFDF91CF910895895F974EFC0135
:1019300060830895FC01E85FF74E8081181614F467
:10194000815080838081811105C08FEF86BB82E04A
:1019500080936F0008951F93CF93DF93BC01FC0128
:1019600020E030E010914B0140E050E0DC01A20F9C
:10197000B31FED01C40FD51F18824F5F5F4F403179
:101980005105B9F7DF01A05FBE4F1D921C92DB012C
:10199000B3951C92D0961C9332966F5F7F4F205F59
:1019A0003F4F211541E03407F9F6FC01E05CFE4FA2
:1019B00011821082329611821082329610823196F4
:1019C000108231962FEF208331962083885B9E4FC3
:1019D000DF91CF911F910C94F420CF93DF93EC0112
:1019E000885B9E4F0E940621CE01DF91CF91B3CF3D
:1019F000FC01EC5BFE4F2081FC01E20FF11DE20FC8
:101A0000F11DE05FFE4F718360830895FC01EC5B84
:101A1000FE4F2081FC01E20FF11DE20FF11DE05F9E
:101A2000FE4F808191810895860F911D860F911D33
:101A3000805F9E4FFC018081918108958E5B9E4F57
:101A4000FC018081918102C0969587956A95E2F7A5
:101A500081700895DF92EF92FF920F931F93CF93BF
:101A6000DF93EC018C010C5B1E4FF801E080F12C40
:101A700089E49BE10E944321EC0EFD1EF701F395E2
:101A80008083F8018081FE01E80FF11DF395D0807D
:101A9000DD20D9F0F801E080F12CFE01EE0DFF1DF4
:101AA000F39560816D1989E49BE10E944921F7015A
:101AB00094E0EE0FFF1F9A95E1F7EC0FFD1FED0D7F
:101AC000F11D31978083DA94E3CFDF91CF911F919D
:101AD0000F91FF90EF90DF90089570E0FC01E60F0A
:101AE000F71FF39524E0660F771F2A95E1F7680F3B
:101AF000791F408189E49BE138CAAF92BF92CF92AF
:101B0000DF92EF92FF920F931F93CF93DF93EC013D
:101B1000FC01EB5BFE4F8081813891F1833809F045
:101B2000ABC089E49BE10E944A0189E49BE10FD8A4
:101B30008DEF9BE10E944E231092111C1092101CFD
:101B40001092131C1092121C10920B1C10920A1C63
:101B500080910C1C90910D1C8E7F90930D1C809396
:101B60000C1C8091241C8F7E8093241C80910E1C61
:101B700090910F1C9F7E90930F1C80930E1C7CC035
:101B80008E010C5B1E4FAA24A394B12CC501F80151
:101B9000008002C0880F991F0A94E2F79093131CEB
:101BA0008093121C90930B1C80930A1C80910E1C36
:101BB00090910F1C906190930F1C80930E1C80914C
:101BC0000C1C90910D1C816090930D1C80930C1C3B
:101BD0008091241C80618093241C89E49BE10E94F5
:101BE0004A0189E49BE13DD8F80160817E01FEEB6A
:101BF000EF1AFEEFFF0A6E0180ECC81A8EEFD80ACA
:101C0000F70180819181F601208131818223932324
:101C1000062E02C0AA0CBB1C0A94E2F78A219B2163
:101C2000892B11F0CE0159DF81E090E0F8010080AE
:101C300002C0880F991F0A94E2F7F60120813181D2
:101C400082239323CA5BDE4F892B31F48DEF9BE116
:101C50000E944A238FEF0FC08DEF9BE10E944E231D
:101C6000F70180819181F801008002C096958795E7
:101C70000A94E2F781708883DF91CF911F910F91D1
:101C8000FF90EF90DF90CF90BF90AF900895FC0150
:101C9000EB5BFE4F208120FD02C021E801C02068DF
:101CA00020832BCFCF93DF93EC01CB5BDE4F3881CA
:101CB000232F217819F022E023272883FC01EA5BF7
:101CC000FE4F208121111FC032974081FC01E40F9B
:101CD000F11DE40FF11DE05FFE4F20813181232BC8
:101CE00091F421E030E002C0220F331F4A95E2F761
:101CF00020953095FC01E05CFE4F4081518124230A
:101D0000352331832083F9DE8881833819F481E01B
:101D10008093091CDF91CF910895FC01EC5BFE4F8D
:101D200020812F3010F42F5F2083E7CEFC01EC5B85
:101D3000FE4F2081222311F021502083DECEFC01B2
:101D4000EC5BFE4F21E030E0008002C0220F331F29
:101D50000A94E2F7329740815181422B532B5183F1
:101D60004083329740815181422B532B51834083D2
:101D7000C4CEFC01EC5BFE4FA08121E030E00A2ED6
:101D800002C0220F331F0A94E2F73297A90140954F
:101D90005095608171814623572351834083329748
:101DA00040815181422B532B51834083FC01EA0F28
:101DB000F11DE05DFE4F2081207F286020839DCEB5
:101DC000FC01EC5BFE4F2081820F911DFC01E05D68
:101DD000FE4F60830895860F911DFC01E05DFE4F6C
:101DE000808108958C5B9E4FFC01808108958F92C5
:101DF0009F92BF92CF92DF92EF92FF920F931F9329
:101E0000CF93DF93FC01E05CFE4F20813181309362
:101E1000F61C2093F51C3296208131813093F81CFA
:101E20002093F71CBC0120E030E009E0D02EAC018B
:101E3000420F531FDA01A05DBE4FDC91D370F90150
:101E4000EB51F34EC081CC7FCD2BC083DC91DC7095
:101E5000C081C37FCD2BC083DC91D295D170C0816E
:101E6000D0FBC4F9C083BC91B07EA081AF71AB2B15
:101E7000A083FB01E05FFE4FA081B181F901EE0F6D
:101E8000FF1FEB53F34EB183A083FA01F39540811A
:101E9000D29EF001D39EF00D1124DF01A85DB34E58
:101EA00055964C9340E050E0E90114E0CC0FDD1F63
:101EB0001A95E1F77F014C018C0E9D1EDA01AA0FE5
:101EC000BB1FFE01EA0FFB1FE80FF91FB0801B2D9F
:101ED0001F70B12EF701E40FF51FEB5CF34EC080CD
:101EE0001C2D107FC12ECB28C082A80DB91D1196C4
:101EF000BC91B295B07FA081AF70AB2BA0834F5F38
:101F00005F4F48305105D1F62F5F3F4F6E5F7F4FD7
:101F10002031310509F08BCFDF91CF911F910F91C7
:101F2000FF90EF90DF90CF90BF909F908F9008959B
:101F3000AF92BF92CF92DF92EF92FF920F931F93D7
:101F4000CF93DF93EC0107DD8091F51C9091F61C97
:101F5000FE01E05CFE4F918380838091F71C90919D
:101F6000F81C329691838083AE0120E030E019E0C6
:101F7000B12ED901AB51B34E7C917370CE01820F5B
:101F8000931FFC01E05DFE4F60816C7F672B6083D7
:101F90007C917C70637F672B60837C9172957170FC
:101FA00070FB64F960837C91707E6F71672B608336
:101FB000F901EE0FFF1FEB53F34E60817181FA01BF
:101FC000E05FFE4F71836083B29EB001B39E700DDF
:101FD0001124FB01E85DF34EE589DC01B395EC9338
:101FE00080E090E06B018901B4E0000F111FBA9509
:101FF000E1F77E01E00EF11EBC01660F771FF601CE
:10200000E80FF91FEB5CF34EA080AA2DAF70AA2E4B
:10201000D801A60FB71FAC0FBD1FAC92E081E295AF
:10202000EF70D701A60FB71F1196EC930196883079
:10203000910511F72F5F3F4F4E5F5F4F2031310504
:1020400009F097CFDF91CF911F910F91FF90EF9003
:10205000DF90CF90BF90AF90089521E030E002C0B4
:10206000220F331F6A95E2F7805C9E4FFC0180814E
:1020700091812823392381E0232B09F480E00895FE
:10208000FC01EC5BFE4F608121E030E0062E02C0D7
:10209000220F331F0A94E2F7209530953497408140
:1020A0005181422353235183408332964081518191
:1020B0004223532351834083462F50E09C01E0E1AB
:1020C0006E9F200D311D1124B90120E030E0FB018D
:1020D000E20FF31F10822F5F3F4F20313105B9F718
:1020E000840F951FFC01F3951082F09610820895DD
:1020F000DC018C9156968C93569711968D919C91FC
:10210000129758969C938E93579783E1FD013396CF
:10211000599601900D928A95E1F70895DC01569643
:102120008C9156978C9357968D919C9158971296B7
:102130009C938E93119783E1FD01799613960190FC
:102140000D928A95E1F70895FC018181928121E049
:1021500030E002C0220F331F6A95E2F728233923AB
:1021600081E0232B09F480E00895CF93C62F81EB03
:102170009BE10E9407216C2F84EC9BE1CF910C9492
:102180000D28CF93C62F81EB9BE10E9421216C2F5C
:1021900084EC9BE1CF910C944129DF92EF92FF9266
:1021A0000F931F93CF93DF938C0181E0F80180831D
:1021B00081EB9BE10E944321E8012396882309F4E7
:1021C0005CC0F80112821182CE010E94F42081EBE2
:1021D0009BE10E944321D82EEE24E394F12CDD20D4
:1021E000F1F0DA946D2D81EB9BE10E944921682F7B
:1021F000CE010E9407216D2D81EB9BE10E944921B8
:10220000F80141815281970102C0220F331F8A9544
:10221000E2F7C901842B952B92838183E0CFCE0115
:102220000E944321F82E84EC9BE10E94EA298F153D
:1022300098F584EC9BE10E94EA29F82ECE010E94D9
:102240004321F81688F46F2DCE010E944921682F92
:10225000CE010E9421216F2DCE010E944921682FBD
:10226000C8018FDFF394EACF84EC9BE10E94EA2956
:10227000682FCE010E9446210FC0CE010E9443214B
:10228000F82EFF2049F0FA946F2DCE010E944921CB
:10229000682FC8016ADFF5CFF80184A5882331F0E3
:1022A0008181928190930B1C80930A1CDF91CF91C6
:1022B0001F910F91FF90EF90DF900895BF92CF9202
:1022C000DF92EF92FF920F931F93CF93DF93EC0176
:1022D0008C010D5F1F4FC8010E944321B82EEE24D0
:1022E000E394F12CBB20E9F085ED9BE10E94E01F17
:1022F0006C01BA946B2DC8010E944921970102C05C
:10230000220F331F8A95E2F7C9018C219D21892B69
:1023100049F76B2DC8010E944921682FCE0131DF9A
:10232000E1CF18828CA5882321F010920B1C10920B
:102330000A1CDF91CF911F910F91FF90EF90DF90DA
:10234000CF90BF900895CF93DF93EC011A8219824A
:10235000188203960E94F420CE01DF91CF91AECF78
:10236000CF93DF93EC0181EB9BE10E94F42084EC9E
:102370009BE10E94F4261092111C1092101CCE01B9
:10238000DF91CF91E0CFCF93DF93EC0103960E94D2
:102390000621CE0149960E94062181EB9BE1909394
:1023A000D21B8093D11BCE01DF91CF91D9CF611188
:1023B00001C084CFF2CECF92DF92EF92FF920F93C3
:1023C0001F93CF93DF93EC01262F2F70D22E809195
:1023D000241C8C7064FF11C08830C9F48091241CC7
:1023E00083708230A1F4622F81EB9BE10E94072170
:1023F00084EC9BE10E94AB2910C0883009F08CC0AE
:102400008091241C8370823009F086C08CC0888142
:10241000811119C06D2DCE01A8DE8091AC02811111
:1024200088C08091AB02813809F083C069817A81CC
:1024300086E691E0DF91CF911F910F91FF90EF9091
:10244000DF90CF90D5CA6D2DCE017EDE8E010D5F5F
:102450001F4F6D2D811142C0C8010E940721C80184
:102460000E944321F82E84EC9BE10E94EA298F15FB
:1024700088F584EC9BE10E94EA29C82EEE24E394BF
:10248000F12CC8010E944321C816E0F46C2DC8014C
:102490000E944921682FCE0174DE6C2DC8010E9474
:1024A000492149815A81970102C0220F331F8A9521
:1024B000E2F7C90180959095842395239A838983B7
:1024C000C394DFCF84EC9BE10E94EA29682FC80106
:1024D0000E9446216D2DCE0148DE06C0C8010E9433
:1024E00021216D2DCE014DDE29813A8181E090E0E0
:1024F00002C0880F991FDA94E2F7822793279A8304
:1025000089838CA5882309F488CF89819A81909347
:102510000B1C80930A1C81CF888181117ECF6D2D89
:10252000CE012FDE7ACF622F81EB9BE10E94212129
:1025300074CFDF91CF911F910F91FF90EF90DF90BB
:10254000CF900895CF92DF92FF920F931F93CF9376
:10255000DF9300D0CDB7DEB78C016B01F42E622F74
:1025600086E691E02A8337DC482F469546954370EE
:102570002A81622F86E691E049832DDC682F637003
:10258000498184EC9BE10E94392720E030E0C0FEC5
:102590000DC0207F832F8F70282BF0FA24F9622F33
:1025A000C8012A83398307DF39812A81D694C794E9
:1025B0003F5F303161F70F900F90DF91CF911F9106
:1025C0000F91FF90DF90CF900895FF920F931F938C
:1025D000CF93DF9381EB9BE10E9443218823D1F0CD
:1025E000F12CC0E0D0E001E010E081EB9BE10E9423
:1025F0004321F81688F46F2D81EB9BE10E9449215D
:10260000980102C0220F331F8A95E2F7C22BD32B09
:10261000F394EBCFC0E0D0E0CE01DF91CF911F91DA
:102620000F91FF90089521E0FC0124A784EC9BE129
:102630000C94112AFC0114A684EC9BE10C94152A3D
:10264000FC011082118220E030E0FC01E20FF31F58
:1026500012822F5F3F4F20323105B9F70895F0CF36
:10266000FC012081E20FF11D62832F5F2F71FC01BD
:1026700020830895FC019181DF01A90FB11D1296FD
:102680008C919F5F9F7191830895FC0181E020816F
:102690009181291301C080E008951F920F920FB617
:1026A0000F9211240BB60F922F933F934F935F938A
:1026B0006F937F938F939F93AF93BF93EF93FF930A
:1026C00080911A1B823019F481ED92E01AD8809122
:1026D0001A1B8350823018F481ED92E02BD9FF91C0
:1026E000EF91BF91AF919F918F917F916F915F918A
:1026F0004F913F912F910F900BBE0F900FBE0F90F7
:102700001F9018951F920F920FB60F9211240BB6BF
:102710000F922F933F934F935F936F937F938F937A
:102720009F93AF93BF93EF93FF9380911A1B8350B6
:10273000823020F481ED92E00E94FB08FF91EF913E
:10274000BF91AF919F918F917F916F915F914F91C9
:102750003F912F910F900BBE0F900FBE0F901F90C7
:1027600018951F920F920FB60F9211240BB60F926D
:10277000EF92FF920F931F932F933F934F935F938B
:102780006F937F938F939F93AF93BF93CF93DF9379
:10279000EF93FF9300B193B18091231C8E3099F495
:1027A00080911A1B8150823070F010E0192B0115B6
:1027B000110511F41092171C89B18F708E3021F120
:1027C00089B18F7021F485ED9BE10E94DD208DEFB2
:1027D0009BE10E94DD21FF91EF91DF91CF91BF91AD
:1027E000AF919F918F917F916F915F914F913F91A9
:1027F0002F911F910F91FF90EF900F900BBE0F90B4
:102800000FBE0F901F9018958091171C8111D8CF83
:10281000C0E0D0E0EE24E394F12CC7010C2E02C0FE
:10282000880F991F0A94E2F780239123892B21F0C6
:102830006C2F81ED92E079D82196C031D10569F7EE
:10284000BFCF1F920F920FB60F9211240BB60F92AB
:102850008F93EF93FF93E1E7F0E080818B7F80839C
:1028600010921C1CFF91EF918F910F900BBE0F9057
:102870000FBE0F901F9018951F920F920FB60F92D8
:1028800011240BB60F922F933F934F935F936F9347
:102890007F938F939F93AF93BF93EF93FF9364992D
:1028A00009C080911C1C81111FC081EC92E00E9424
:1028B0006B241AC080911B1C811116C081EC92E020
:1028C0000E94672381E080931C1C809171008460CA
:1028D0008093710080919400909195008A5B9F4F46
:1028E00090939B0080939A00FF91EF91BF91AF91DD
:1028F0009F918F917F916F915F914F913F912F9118
:102900000F900BBE0F900FBE0F901F901895CF9396
:10291000DF938091231C813129F410920D1C1092B9
:102920000C1CD7C0C091241CC295C170D091231C2F
:1029300084EC9BE10E94FE29D15041E050E09A01D5
:1029400002C0220F331FDA95E2F783708F5F02C057
:10295000440F551F8A95E2F7242B352B2C2B3093EF
:102960000D1C20930C1C8091091C882359F0809128
:102970000C1C90910D1C817F90930D1C80930C1C5E
:102980001092091C8091231C8A3049F480910C1C00
:1029900090910D1C817F90930D1C80930C1C809155
:1029A000241C807EB9F18091231C893041F08091F4
:1029B000231C8A3021F08091231C8C3099F4609183
:1029C000241C629566956770653031F48091231CF4
:1029D000893009F06FC065E06C5F41E08DEF9BE1ED
:1029E0000E94CE218091231C8E30A1F480911A1B6D
:1029F000843039F0853041F0833061F441E068E0A3
:102A000005C041E067E002C041E061E08DEF9BE17D
:102A10000E94CE218091CE02882331F080910E1C3D
:102A200090910F1C906405C080910E1C90910F1C1A
:102A30009F7B90930F1C80930E1C8091231C8D30E4
:102A4000A1F48091AB02813881F48091AC028F3F78
:102A5000C1F50BC0813049F480910C1C90910D1C84
:102A6000916090930D1C80930C1C8091231C8A30E4
:102A700081F58091D002882349F080910C1C9091BF
:102A80000D1C846090930D1C80930C1C8091CF02D0
:102A9000882331F080910C1C90910D1C886005C03A
:102AA00080910C1C90910D1C826090930D1C809362
:102AB0000C1C0FC08091231C8C3009F48CCF64E077
:102AC0008BCF8111C7CF80910C1C90910D1C94600D
:102AD000C8CFDF91CF910895BF92CF92DF92EF924E
:102AE000FF920F931F93CF93DF9300D01F92CDB728
:102AF000DEB78091FC1C9091231C913109F4F4C441
:102B000090E0FC013197EF30F10508F02DC3E45B54
:102B1000FF4F0C945D2E8091231C8C3089F18091A5
:102B2000231C8E3069F18091231C8F3049F18091F4
:102B3000231C8D3029F18091CE02811121C080911A
:102B4000241C8295817091E089279091241C80FB40
:102B500094F99093241C8091231C8B3039F460915C
:102B6000241C629561708CE19BE121DC8091231C27
:102B7000893009F41EC38091231C8A3009F419C3DB
:102B80008091231C8E3009F0EFC280911A1B843093
:102B900059F0853021F0833009F0E6C205C081ED9F
:102BA00092E00E941F0CE0C281ED92E00E94FA0BBD
:102BB000DBC28091CE0281111DC08091231C8A301E
:102BC000C9F08091231C8D3009F4FCC28091241C33
:102BD000837081F08091241C8C7F8093241C9091C1
:102BE000251C9370990F990F8091241C837F892B4A
:102BF0008093241C8091231C8A3009F0B5C2109266
:102C0000CF02B2C28091CE0281111EC08091231CDE
:102C10008A30D1F08091231C8D30B1F08091241C3A
:102C20008370813089F08091241C8C7F8160809337
:102C3000241C9091261C9370990F990F8091241C4D
:102C4000837F892B8093241C8091231C8A3009F078
:102C50008BC28091D00291E089278093D00284C2F8
:102C60008091CE0281111FC08091231C8A30D9F03F
:102C70008091231C8D3009F4B6C28091241C83708E
:102C8000823089F08091241C8C7F82608093241C88
:102C90009091271C9370990F990F8091241C837F2A
:102CA000892B8093241C8091231C8A3009F05CC2FC
:102CB00081E08093CF0258C28091CE02811154C22C
:102CC0008091241C8F71806208C08091CE02811196
:102CD0004BC28091241C8F7180648093241C81E0FE
:102CE0008093161C41C28091CE0281113DC2809119
:102CF0001D1C81115AC08091231C8E30C1F580911A
:102D00001A1B8430A1F1823071F581E08093171C89
:102D10008CE19BE15ADC7C01009729F1B12C00E0A9
:102D200010E0CC24C394D12C9601002E02C0220FB7
:102D3000331F0A94E2F72E213F21232B79F08B2DAC
:102D4000807FB82E802F8F70B82A6B2D8CE19BE18D
:102D500032DB6B2D81ED92E00E941E0B0F5F1F4F47
:102D60000031110509F781ED92E00E94AE0B8091D0
:102D7000231C8D3069F48091AB02813809F0F4C1D5
:102D80008CE19BE1EDDA86E691E00E94960E5CC054
:102D90008091241C8F718066A0CF8091CE0281111A
:102DA000E3C180911D1C882319F010921D1CDCC109
:102DB0008091231C8E30C1F580911A1B8330A1F1C4
:102DC000823071F581E08093171C8CE19BE1FDDB83
:102DD0007C01009729F1B12C00E010E0CC24C394D1
:102DE000D12C9601002E02C0220F331F0A94E2F765
:102DF0002E213F21232B79F08B2D807FB82E802F21
:102E00008F70B82A6B2D8CE19BE1D5DA6B2D81EDAB
:102E100092E00E941E0B0F5F1F4F0031110509F752
:102E200081ED92E00E94D80A8091231C8D3071F5CB
:102E30008091AB02813809F097C18CE19BE190DA77
:102E400086E691E00E948D0E8091AC02882349F0C5
:102E500060E08CE19BE1ABDA86E691E00E947D0DBB
:102E600083C161E08CE19BE1A2DA86E691E00E94F9
:102E7000F20E282F86E691E02B830E94060DBC01FE
:102E80002B8141E08CE19BE15DDB6EC18091241CD4
:102E90008F71806822CF8091CE02811165C18091AF
:102EA000241C807E31F48091241C8F71806A809371
:102EB000241C8091231C8E3021F481ED92E00E942D
:102EC0000F0C8091231C8B3019F48CE19BE110D9FD
:102ED0008091231C893039F48091241C8F71806A81
:102EE0008093241C41C18091231C8A3061F489E4C1
:102EF0009BE10E94970889E49BE10E94310689E4E6
:102F00009BE10E94A7058091231C8D3009F07CC1B4
:102F10008091AB02813809F077C186E691E00E948A
:102F20009F0E8CE19BE11CDA60E0E0C18091CE0253
:102F300081111AC18091231C8D3009F0F1C080915C
:102F4000AB02813809F0ECC0CFC28091CE02811172
:102F50000BC18091231C8E3021F481ED92E00E9400
:102F60000F0C8091231C893041F08091231C8A3002
:102F700021F08091231C8C30B1F48091231C893086
:102F800009F0B0C189E49BE10E94970889E49BE1C4
:102F90000E94310689E49BE10E94A7058091241CD0
:102FA0008F7E8093241C8091231C8D3009F0A2C158
:102FB0008091AB02813809F09DC186E691E00E94C4
:102FC000B90E61E093C18091CE028111CDC0809194
:102FD000231C8D3009F0A6C18091AB02813809F025
:102FE000A1C182C28091CE028111BEC08091231CFA
:102FF0008B3019F48CE19BE17BD88091231C8E30BF
:1030000021F481ED92E00E940F0C8CE19BE1A8D9A4
:103010008091231C8D30B1F18091231C893009F4FB
:10302000D3C18091231C8C3009F4CEC18091231C24
:103030008A3009F4C9C18DE08093231C62E089E4E1
:103040009BE10E949B0584EC9BE10E94FA2986E6A5
:1030500091E00E94470E10E000E0612F86E691E0CB
:103060000E942D10811101E01F5F1031B1F7809196
:10307000AB02813839F5002329F186E691E00E9400
:10308000520E20C086E691E00E94520E8091AB0263
:103090008138C1F48091AC02811114C061E08CE1EF
:1030A0009BE185D986E691E00E94F20E282F86E604
:1030B00091E02B830E94060DBC012B8141E08CE145
:1030C0009BE140DA80910A1C90910B1C9A838983C2
:1030D00089819A8190930B1C80930A1C00CE809169
:1030E000CE02811141C08091231C8B3021F48CE1F0
:1030F0009BE10E9478108091231C8D3009F06DC1F6
:103100008091AB02813809F068C1EEC18091231C27
:103110008E3051F18091231C8B3009F081C124C085
:103120008091231C8B3021F48CE19BE10E9478106C
:103130008091231C8E3021F481ED92E00E940F0CCF
:103140008091231C893009F4BCC08091231C8C30F1
:1031500009F4B7C08091231C8D3009F4B2C080916E
:10316000231C8A3009F080C08091231C8D3009F027
:10317000A4C18091AB02813809F09FC186E691E03D
:103180000E94F20E682F86E691E00E94EB0E482F17
:1031900046954695437086E691E04B830E94F20E79
:1031A000682F86E691E00E94EB0E682F63704B81DA
:1031B00096C16091241C6295617089E49BE10E9434
:1031C000CD06DECC8091AB02813809F013CD809121
:1031D000AC02813009F00ECD60914C0186E691E0A1
:1031E0000E94E00E07CD8091AB02813809F05BCDE3
:1031F0008091AC02813009F056CD60914D0186E698
:1032000091E00E94E00E4FCD60E089E49BE10E94D6
:103210009B058091241C8F7E8093241C8CE19BE174
:103220009FD884EC9BE10E94FA2989E49BE10E94EB
:10323000A108882351F08091241C80618093241C74
:1032400089E49BE10E9431060DC08091241C8F7E91
:103250008093241C89E49BE10E94310689E49BE170
:103260000E94A70589E01CC061E089E49BE10E94FF
:103270009B058CE19BE174D884EC9BE10E94FA29C8
:1032800089E49BE10E94A108882369F08091241CB5
:1032900080618093241C89E49BE10E9431068AE0CE
:1032A0008093231C1CCD8091241C8F7E8093241C32
:1032B00089E49BE10E94310689E49BE10E94A70515
:1032C000EECF8091231C893021F489E49BE10E9498
:1032D000970889E49BE10E94310689E49BE10E9402
:1032E000A7053DCF8A3009F44DCE50CE8CE19BE14D
:1032F0005ED83ACF8CE19BE133D86091241C629573
:1033000061708CE19BE153D884EC9BE10E94FA2927
:103310008BE08093231C8CE19BE10E948E10109225
:10332000161C22CF8091231C8B3021F48CE19BE171
:103330000E9478108091231C8E3021F481ED92E060
:103340000E940F0C8091231C893021F489E49BE1B9
:103350000E9431068091231C8A3069F18091231CE0
:103360008D3049F160E089E49BE10E949B058091EA
:10337000231C8C3091F089E49BE10E9431068CE1A2
:103380009BE10E94B01184EC9BE10E94F6298CE045
:103390008093231C81E08093161C8091241C8F7ED7
:1033A0008093241C1092111C1092101C10920B1C64
:1033B00010920A1CD9CE89E49BE10E94310689E46F
:1033C0009BE10E94A705CECF89E49BE10E943106D4
:1033D00089E49BE10E94A7052ECE8091231C8E30AC
:1033E00009F4C2CE8091241C8F7E8093241C89E432
:1033F0009BE10E94A70560E089E49BE10E949B0598
:103400008EE08093231C8CE19BE10E94B01184EC40
:103410009BE10E94FA2981ED92E00E942A0CA4CE41
:103420008091CE0281111DC08091231C893021F032
:103430008091231C8A3081F489E49BE10E949708E3
:1034400089E49BE10E9431068091241C84FD04C024
:1034500089E49BE10E94A70581EC92E00E94272469
:1034600083CE81EC92E00E943E248091231C8C301C
:1034700009F47ACE89E49BE106D7811106C089E47C
:103480009BE10E94A108882351F08091241C806157
:103490008093241C89E49BE10E94310665CE8091D3
:1034A000241C8F7E8093241C89E49BE10E943106BA
:1034B00089E49BE10E94A70557CE8091231C8D30A3
:1034C00031F48091AB02833811F421DA0DC04091C0
:1034D000241C4695469543706091241C637084ECCF
:1034E0009BE10E943927F1CF0F900F900F90DF9151
:1034F000CF911F910F91FF90EF90DF90CF90BF90F1
:103500000895F89412B811B815B814B88FEF87B9A8
:103510001BB890EF9AB998E39EB99FEE9DB980BB16
:1035200080E090E890930D1C80930C1C8BB1806F11
:103530008BB97298759A1092001D1092FF1C109210
:10354000FE1C1092011D1092031D1092021D10927C
:10355000FD1C8091AB02813821F486E691E00E9447
:10356000520E8DEF9BE1F1D68BED9BE169D885ED95
:103570009BE120D584EC9BE10E94F42681EB9BE14A
:1035800033D689E49BE10E94F3008CE19BE10E9429
:10359000A3118CE19BE10E94B01181ED92E00E94A9
:1035A000B90881EC92E00E94572386E691E00E94E0
:1035B000AB0C8BED9BE19093DA1B8093D91B84EDD0
:1035C000E8E2FCE1DF011D928A95E9F78BE0809348
:1035D000231C8093FC1C80DA8091241C8C7F8093B8
:1035E000241C8091241C837F8093241C4091241CE4
:1035F0004695469543706091241C637084EC9BE172
:103600000E9439278091241C8F7180688093241C2C
:103610008091241C8F7E8093241C1092251C109274
:10362000261C1092271C1092221C1092211C84EC44
:103630009BE10E94FA2989E49BE10E949305109284
:103640001F1C10921E1C10921D1C61D910921C1C74
:1036500010921B1C10921A1C1092191C1092181C0C
:103660001092171C89E49BE10E94AE088CE19BE15B
:103670000E9413131092B00082E08093B10081E0A9
:10368000809370001092900095E0909391001092BA
:10369000710095E59093690080936A008FE18DBB7E
:1036A0008DEF9BE1A6D7789408951F920F920FB6E5
:1036B0000F9211240BB60F922F933F934F935F936A
:1036C0006F937F938F939F93AF93BF93EF93FF93EA
:1036D000809171008D7F8093710089B18F7071F03E
:1036E00029B12F708091FD1C30E090E02817390738
:1036F00031F48091FD1C8093FC1C01C0EDD9FF9139
:10370000EF91BF91AF919F918F917F916F915F9159
:103710004F913F912F910F900BBE0F900FBE0F90C6
:103720001F90189589B18F70B1F089B18F70809317
:10373000FD1C89B18F708C3071F48091241C8061E4
:103740008093241C8091231C8C3021F489E49BE11C
:103750000E943106DCD88091940090919500875F9B
:103760009C4F9093990080939800809171008260A3
:103770008093710008951F920F920FB60F9211243B
:103780000BB60F922F933F934F935F936F937F935B
:103790008F939F93AF93BF93EF93FF93C3DFFF91FB
:1037A000EF91BF91AF919F918F917F916F915F91B9
:1037B0004F913F912F910F900BBE0F900FBE0F9026
:1037C0001F9018951F920F920FB60F9211240BB6EF
:1037D0000F922F933F934F935F936F937F938F93AA
:1037E0009F93AF93BF93EF93FF939CDFFF91EF9174
:1037F000BF91AF919F918F917F916F915F914F9109
:103800003F912F910F900BBE0F900FBE0F901F9006
:1038100018951F920F920FB60F9211240BB60F92AC
:103820002F933F934F935F936F937F938F939F93C8
:10383000AF93BF93EF93FF9375DFFF91EF91BF912C
:10384000AF919F918F917F916F915F914F913F9138
:103850002F910F900BBE0F900FBE0F901F901895D9
:103860001F920F920FB60F9211240BB60F922F9347
:103870003F934F935F936F937F938F939F93AF93F8
:10388000BF93EF93FF934EDFFF91EF91BF91AF9105
:103890009F918F917F916F915F914F913F912F9168
:1038A0000F900BBE0F900FBE0F901F901895CF92E8
:1038B000DF92FF920F931F93CF93DF931F92CDB7A9
:1038C000DEB7F82E2091241C23709091291C9C7F38
:1038D000922B9093291C2091241C2C709091291CD0
:1038E000937F922B9093291C9091241C9295917018
:1038F0008091291C90FB84F98093291C2091241C21
:10390000207E9091291C9F71922B9093291C89E411
:103910009BE10E94DB0786E691E00E94F70E81ECB6
:1039200092E00E946B268FEFF89E60011124E0E187
:10393000CE0ED11C08E21CE1F80161918F01C60195
:1039400069830E94F82E6981681719F0C6010E94E8
:10395000002FFFEFCF1ADF0A8CE10C3F180761F749
:1039600010921F1C41E04F0D68E08DEF9BE10F901E
:10397000DF91CF911F910F91FF90DF90CF9091C673
:10398000CF931092071C89B18F70883009F043C023
:1039900081EB9BE129D489E49BE10E94F3008CE157
:1039A0009BE10E94A3118CE19BE10E94B01181ED8B
:1039B00092E00E94B90881EC92E079D686E691E027
:1039C0000E94AB0CF894729A7598C0E08C2F6FDF50
:1039D0008BB18F709C2F9295907F892B8BB9109211
:1039E000FF1C8091FF1C8F3F91F01092FE1C809174
:1039F000FE1C843630F48091FE1C8F5F8093FE1C89
:103A0000F6CF8091FF1C8F5F8093FF1CEACFCF5FC2
:103A1000C031E1F678948091231C8B3089F038F422
:103A2000893009F44FC08A3009F44CC077C08D301A
:103A300009F44DC008F446C08E3009F45CC06EC075
:103A400089B18F708B3069F581E18093231C80915F
:103A5000241C83608093241C8091241C837F80938A
:103A6000241C8091241C8F7E8093241C8091241C14
:103A70008F718093241C4091241C46954695437079
:103A80006091241C637084EC9BE10E94392781E0E3
:103A90008093161C87E090E090930B1C80930A1C87
:103AA0003BC08CE19BE10E94A3118CE19BE10E9451
:103AB000B0116091241C629561708CE19BE10E94C1
:103AC000D7112AC089E49BE10E94AA0825C08091F1
:103AD000AB02813839F0833809F589E49BE10E9413
:103AE000AA081CC086E691E00E94401086E691E09C
:103AF0000E947D0D13C089B18F708E3049F481ED25
:103B000092E00E94B90881ED92E00E942A0C04C064
:103B100081ED92E00E94550C0E9487148091CE02A4
:103B2000882339F081EC92E00E949A26CF910C9480
:103B30008714CF910895FF920F931F93CF93DF9334
:103B4000F82E08E21CE1C0E1D0E0C852DC418FEF62
:103B5000F89EC00DD11D1124CE01800F911F0E942F
:103B6000F82EF80181938F01FCE10C3F1F07A1F7AC
:103B70002091291C23709091241C9C7F922B909360
:103B8000241C2091291C2C709091241C937F922B33
:103B90009093241C9091291C929591708091241CE3
:103BA00090FB84F98093241C2091291C207E909105
:103BB000241C9F71922B9093241C84EC9BE10E9407
:103BC000F4268CE19BE10E94B01189E49BE10E9404
:103BD000300886E691E00E94980F81EC92E00E9406
:103BE00084266091241C629561708CE19BE10E94A7
:103BF000D7118BE08093FC1C10921E1C41E04F0DEE
:103C000067E08DEF9BE14DD5DF91CF911F910F9133
:103C1000FF900C946C151F93CF93DF931F92CDB739
:103C2000DEB780911E1C882321F080911E1C8150DC
:103C300082DF80911F1C882321F080911F1C8150FE
:103C400036DE8091061C813009F45BDC8091071C14
:103C5000813009F495DE8BED9BE10E9445138823AA
:103C600009F47AC18BED9BE10E943A13682F80938F
:103C7000201C8091CE02882351F064FF6DC16F70CB
:103C800081EC92E00F90DF91CF911F91FFC5809161
:103C90001A1B8150823020F481ED92E00E941E0BAD
:103CA0008091231C8B3021F08091231C8E30A1F455
:103CB0008091231C8E3029F480911A1B853009F4E1
:103CC000BEC08091231C8E3009F4C3C06091201CBB
:103CD0008CE19BE10E94DB118091231C8D3009F067
:103CE0006DC08091AB02813811F58091AC028823C0
:103CF00019F0813041F062C06091201C8CE19BE1A1
:103D00000E94DB115BC08091201C682F6F7084FFC4
:103D100005C089E49BE10E94EA0604C089E49BE1B6
:103D20000E94E30186E691E00E942A0D47C0833895
:103D300009F044C06091201C6F7086E691E00E94FB
:103D40002D108823D9F18091201C682F6F7084FF7B
:103D5000A1C0162F8EEA92E05AD28EEA92E093D258
:103D6000823008F4A6C061E08EEA92E092D28F3FE2
:103D700009F49FC08FEF8093AD0289E49BE10E941C
:103D8000A70589E49BE10E944A018CE19BE10E9426
:103D9000B01140910C1C50910D1C5E7F50930D1C76
:103DA00040930C1C40910C1C50910D1C417F509372
:103DB0000D1C40930C1C1F3F09F07BC08091231CFD
:103DC0008C30D1F48091241C84FD07C06091201CAC
:103DD0008CE19BE10E94DB110FC08091201C682FB9
:103DE0006F7084FF05C089E49BE10E94EA0604C06D
:103DF00089E49BE10E94E3018091231C8A3021F039
:103E00008091231C893061F48091201C682F6F7091
:103E100084FF9DC089E49BE10E94EA068091231CF7
:103E20008091231C813109F097C06091201C8CE1A6
:103E30009BE10F90DF91CF911F910C94DB1185EDE9
:103E40009BE1BED0892B09F03CCF89B18F7081F006
:103E500038CF80911A1B833009F038CF85ED9BE174
:103E6000AFD0892B09F432CF89B18F7041F02ECFBA
:103E700081ED92E00E941F0C0E94871422CF81EDF9
:103E800092E00E94FA0B8CE19BE10E94B0110E942B
:103E900087141CCF8EEA92E0D4D18EEA92E0F3D15F
:103EA000882309F452C060E08EEA92E0F2D1182F24
:103EB00061CF612F86E691E00E941E0D882359F1A3
:103EC000813009F07BCF8093AD0289E49BE10E94B1
:103ED0003106612F86E691E00E94EB0E482F469551
:103EE00046954370612F86E691E049830E94EB0E70
:103EF000682F6370498184EC9BE1BBD7612F86E614
:103F000091E00E946D0D0E94871480910C1C90918D
:103F10000D1C916015C01092AD02612F86E691E0F4
:103F20000E94140D212F41E0BC018CE19BE10E9415
:103F3000A2120E94871480910C1C90910D1C946019
:103F400090930D1C80930C1C39CF1FEF13CF89E485
:103F50009BE10E94E30162CF0F90DF91CF911F910F
:103F600008958DEF9BE10AD28BED9BE10E942F1308
:103F700085ED9BE119D084EC9BE153D781EB9BE16C
:103F800045D189E49BE10E9433018CE19BE10E94D1
:103F9000C31181ED92E00E94F00881EC92E096D38B
:103FA00086E691E00C94ED0CFC01118210821382E4
:103FB00012820895FC0111821082138212820895E8
:103FC00080B123B190E0922B0895CF92DF92EF92CF
:103FD000FF920F931F93CF93DF9300D000D01F92D7
:103FE000CDB7DEB77C01FC01228133813C832B837A
:103FF00080819181822793279A838983DD24D394BA
:1040000000E010E0CC24C39489819A8180FFB5C080
:10401000402F4F708B819C81817029B12F7030E0CF
:104020002430310509F459C03CF42230310579F0CF
:104030002330310579F192C0952F907F27303105DB
:1040400009F472C02830310509F47AC087C0013004
:10405000110559F00230110569F00115110509F03B
:104060008CC08091241C837F09C08091241C837F95
:10407000846004C08091241C837F88608093241C0A
:104080008091241C8695869583708093251C4D2DE8
:1040900062E045C00130110559F00230110569F0A8
:1040A0000115110509F069C08091241C837F09C0A6
:1040B0008091241C837F846004C08091241C837FB2
:1040C00088608093241C8091241C8695869583703B
:1040D0008093261C4D2D63E022C00130110559F05C
:1040E0000F30110569F00115110509F046C08091E6
:1040F000241C837F09C08091241C837F846004C0BA
:104100008091241C837F88608093241C8091241CD0
:104110008695869583708093271C4D2D64E08DEFE6
:104120009BE15D83BED228C0592F542B80FB54F9EC
:104130005F7D5F7B5F7754FD20C0D0921E1C0BC05B
:10414000592F542B80FB54F95F7D5F7B5F7754FDC3
:1041500014C0D0921F1CC0921D1C0FC0507F542B46
:1041600080FB54F95F7D5F7B5F77652FF70184816A
:1041700095815D830E9430135D8189819A81969536
:1041800087959A8389838B819C81969587959C835B
:104190008B830F5F1F4FD394F1E1DF1235CF0F9068
:1041A0000F900F900F900F90DF91CF911F910F9173
:1041B000FF90EF90DF90CF900895CF93DF93EC01C5
:1041C00080B123B190E0922B9B838A83288139812F
:1041D0008217930711F0CE01F8DE8A819B819983C3
:1041E0008883DF91CF910895FC01128A20E030E0AE
:1041F0004FEFFC01E20FF31F40832F5F3F4F203151
:104200003105B9F720E1FC01218B0895EDCFFC01C8
:10421000928981899817A0F482898F5F828B228985
:10422000222369F0822F90E0DC011197AE0FBF1FAF
:104230003C91DF01A80FB91F3C932150F1CF60835F
:104240000895FC0120E082892817E0F4DF01A20F25
:10425000B11D8C91861314C0322F8289381768F4EF
:10426000832F90E0DC011196AE0FBF1F4C91DF0150
:10427000A80FB91F4C933F5FF0CF82898150828B8A
:104280002F5FE1CF0895FC0182890895FC01628BC4
:104290000895860F911DFC0180810895FC018081A5
:1042A0000895FC0190E080E02289921748F4DF0134
:1042B000A90FB11D2C91821708F48C919F5FF4CF48
:1042C0000895FC0190E080E12289921748F4DF0113
:1042D000A90FB11D2C91281708F48C919F5FF4CF82
:1042E0000895FC01759B30C075986D98659B05C05D
:1042F00086819781019697838683659B05C0868119
:104300009781019697838683659902C017821682EA
:104310006D9A759A868197810B9720F08681978197
:10432000449758F086819781893E934068F081E0F8
:104330008187128617821682089581E0828784E140
:1043400090E097838683EECF0895FC011382168652
:104350001586148A138A168A158A108E178A108A6F
:104360001786128A118A1582118612861782168282
:10437000138610821182128214860895E6CFFC0102
:1043800087859089411105C0609570958623972394
:1043900002C0862B972B908B87870895662351F058
:1043A0002FEF260F61E070E002C0660F771F2A959D
:1043B000E2F702C06FEF7FEFE2CFCF93DF93EC0124
:1043C0008B8181118EC08C818F5F8C838C81803832
:1043D00009F41C828C8181110AC0888591E08927AB
:1043E00088878881882319F0888181508883759A0D
:1043F000729A9D819295907F8BB18F70892B8BB92A
:1044000049895A892D8181E090E0BC0102C0660F84
:10441000771F2A95E2F79B0124233523232B31F0C4
:10442000888580FF729A80FD72980DC02F8538892B
:104430004D8102C0880F991F4A95E2F7822393238A
:10444000892B09F072988B85882381F08D818830C3
:1044500029F4888580FF729A80FD72988D818A3058
:1044600029F4888580FD729A80FF72984D855E855B
:104470002B893C896D8181E090E002C0880F991FF3
:104480006A95E2F7242B352B82239323892B09F09D
:1044900075984D895E892D8181E090E0BC0102C054
:1044A000660F771F2A95E2F79B0124233523232BE0
:1044B000B1F0288520FF759A20FD75984D855E85A1
:1044C0002B893C896D8102C0880F991F6A95E2F79C
:1044D000242B352B82239323892B09F07598CE0149
:1044E00000DF8B81823009F047C08091231C81312D
:1044F00081F42B893C894D8181E090E002C0880FD6
:10450000991F4A95E2F782239323892B09F469C006
:104510000FC02D853E854D8181E090E002C0880F5F
:10452000991F4A95E2F782239323892B09F059C0FA
:10453000898D882309F455C04D895E892D8181E0DC
:1045400090E0BC0102C0660F771F2A95E2F79B013D
:1045500024233523232B81F04B895C892D853E85CF
:104560006D8102C0880F991F6A95E2F7242B352BC5
:1045700082239323892BB9F58881882301F12D812A
:10458000898130E090E001972817390741F488814C
:10459000843009F472988881823009F4729A2D81EE
:1045A0008A8130E090E001972817390741F488812B
:1045B000833009F475988881813009F4759A8B816C
:1045C000873031F48D818F5F8D838D818F708D83E6
:1045D0008B818F5F8B838B8187708B83DF91CF91F2
:1045E0000895759AA9CF888580FF759A80FD759882
:1045F000C3CFCF93DF9300D01F92CDB7DEB77298B1
:10460000759A1B828B818031D8F49B819295907F23
:104610008BB18F70892B8BB91A828A818F3F61F0A1
:1046200019828981843620F489818F5F8983F9CF4B
:104630008A818F5F8A83F1CF8B818F5F8B83E2CFFB
:10464000729A75981B822FE08B818031E8F48B8100
:10465000922F981B9295907F8BB18F70892B8BB97D
:104660001A828A818F3F61F019828981843620F411
:1046700089818F5F8983F9CF8A818F5F8A83F1CFA8
:104680008B818F5F8B83E0CF0F900F900F90DF9126
:10469000CF91089521E0FC0123870895FC01138642
:1046A0000895FC0184E08083618342830895FC01C6
:1046B00080E180878FEF9FEF978386831186128634
:1046C000138614861586178616860895F0CFCF9325
:1046D000DF93EC018091231C8A3049F018F4893073
:1046E00059F052C08C3079F18D30B1F14DC07098D5
:1046F00071987698779848C060E089E49BE10E94C1
:104700001502682F6F708CE19BE10E94DB118D8593
:10471000811110C060E089E49BE10E94150221E054
:1047200030E002C0220F331F8A95E2F730930B1C52
:1047300020930A1C709932C0719930C076992EC0AE
:1047400077992CC021C077988D8581111DC08091EB
:10475000241C84FD28C018C08091AB02813819F454
:104760008091AC0204C0833879F48091AD0281302D
:1047700059F460E089E49BE10E941502682F6F7094
:104780008CE19BE10E94DB118D858823E9F08E810D
:104790009F819093111C8093101C16C08CE19BE1AB
:1047A0000E94B011F1CF60E089E49BE10E94150204
:1047B00021E030E002C0220F331F8A95E2F73093E8
:1047C0000B1C20930A1CE0CFDF91CF910895CF936B
:1047D000DF93EC018CE19BE10E941A1389E49BE1D9
:1047E0000E94B40880910C1C90910D1C99838883C1
:1047F00080910A1C90910B1C9B838A838091101CD2
:104800009091111C9D838C83DF91CF910895CF935C
:10481000DF93EC018CE19BE10E94131389E49BE19F
:104820000E94AE088881998190930D1C80930C1C86
:104830008A819B8190930B1C80930A1C8C819D81A3
:104840009093111C8093101CDF91CF910895CF930A
:10485000DF93EC01BCDF21E02093161C10920B1CAF
:1048600010920A1CE0E1FCE1118210828E819F818E
:10487000918380832D87DF91CF910895CF93DF932C
:10488000EC01C5DF1D86DF91CF91089521E030E076
:1048900002C0220F331F6A95E2F7FC01468157815F
:1048A00024273527378326833093111C2093101C2F
:1048B0000895FC0181858F5F8F70818782858F5F6E
:1048C0008F70828783858F5F8F70838784858F5FEA
:1048D0008F7084870895DF92EF92FF920F931F935A
:1048E000CF93DF93EC01709951C171994FC17699C3
:1048F0004DC176994BC189E49BE10E94B407809138
:10490000231C8A3061F020F4893009F4C5C02CC121
:104910008C3009F4DCC08D3009F4F4C025C18F85DA
:10492000882349F189E49BE1AEDC19858130C9F027
:10493000833059F560E089E49BE1ABDC810F8F7037
:104940008A87198561E089E49BE1A3DC810F8F7080
:104950008B87198562E089E49BE19BDC810F8F7076
:104960000DC060E089E49BE194DC810F8F708A8741
:1049700099859B8703C089858A878B878C8700E010
:1049800010E0EE24E394F12C27C01A871B871C87C4
:10499000F6CF89E49BE177DC8130A9F178F5D1107D
:1049A0003EC06091241C62956695677040E089E482
:1049B0009BE10E941F0460E089E49BE10E941502D4
:1049C0008F7098B1907F982B98B9709A0F5F1F4F96
:1049D0000430110509F449C0D02EFE01E00FF11F8B
:1049E000C701018402C0880F991F0A94E2F72E8143
:1049F0003F8182239323892B49F3CBCF823079F2F5
:104A0000833019F00CC001FD0AC06091241C62952E
:104A100066956770402F89E49BE10E941F0442E085
:104A2000D41679F053E0D516B1F081E0D812C3CF97
:104A300089E49BE128DC80FDACC08E858111A9C092
:104A4000C5CF89E49BE11FDC833009F4AFC08E85BC
:104A50008111ACC0BBCF89E49BE115DC833009F444
:104A6000B1C08E858111AEC0B1CF8D85811104C0DA
:104A700010920B1C10920A1CF12C01E010E08D85A5
:104A8000811105C089B18F708A3009F0A8C0F394F4
:104A900044E0F412F4CF68C081E090E0098402C0E1
:104AA000880F991F0A94E2F72E813F818223932376
:104AB000892B09F459C089E49BE1E5DB8111A6C08B
:104AC0008091241C807E803A09F0A0C0FCC081E067
:104AD00090E0098402C0880F991F0A94E2F72E81A2
:104AE0003F8182239323892B09F43EC089E49BE113
:104AF000CADB8111BAC08091241C807E803A09F003
:104B0000B4C0E1C081E090E0098402C0880F991F21
:104B10000A94E2F72E813F8182239323892B21F18E
:104B20008091AB02813819F48091AC0204C08338C3
:104B3000D9F48091AD028130B9F489E49BE1A3DB23
:104B4000882309F4C0C065E089E49BE10E94ED047C
:104B500060E089E49BE10E941502682F6F7060613C
:104B60008CE19BE10E94DB118D85882331F08E81E1
:104B70009F819093111C8093101CCE01DF91CF91E7
:104B80001F910F91FF90EF90DF9093CECE019FDDAC
:104B9000B2CE61E089E49BE10E9415028295807F9C
:104BA00098B19F70982B98B9719A10CF62E089E400
:104BB0009BE10E9415028F7091B3907F982B91BB5F
:104BC000769A04CF63E089E49BE10E941502829506
:104BD000807F91B39F70982B91BB779AF7CE6F2D02
:104BE00089E49BE10E94150220910A1C30910B1C64
:104BF000A80102C0440F551F8A95E2F7CA01822B13
:104C0000932B90930B1C80930A1C41CF6091241C22
:104C100062956695677089E49BE10E94ED0460E00F
:104C200089E49BE10E941502682F6F7060618CE13E
:104C30009BE10E94DB118D85811196CF60E089E4B4
:104C40009BE10E94150240910A1C50910B1C21E02F
:104C500030E002C0220F331F8A95E2F7242B352B58
:104C600030930B1C20930A1C7FCF6091241C62950B
:104C70006695677089E49BE10E94ED0460E089E439
:104C80009BE10E9415028295807F91B39F70982BC3
:104C900091BB8D85811104C08091241C84FD02C0CC
:104CA000779A62CF60E089E49BE10E94150221E0DF
:104CB00030E002C0220F331F8A95E2F730930B1CBD
:104CC00020930A1CEDCFDF91CF911F910F91FF90A0
:104CD000EF90DF900895DC0116968D919C911797C7
:104CE0009093FA1C8093F91C1F969C911F97EBEFF1
:104CF000FCE1808190FB80F980831E969C918081ED
:104D000090FB81F980830895CF93DF93EC01CFDC92
:104D10008091F91C9091FA1C9F838E83EBEFFCE14C
:104D2000808181708F878081869581708E87DF91E9
:104D3000CF9108952FEF3FEFFC013783268308952D
:104D4000413051F028F0423071F0433081F0089545
:104D50006F7088B1807F04C06295607F88B18F706A
:104D6000862B88B908956F7081B3807F04C06295E7
:104D7000607F81B38F70862B81BB0895413059F0DD
:104D800028F0423069F0433081F0089560FD709A58
:104D900060FF7098089560FD719A60FF71980895A2
:104DA00060FD769A60FF7698089560FD779A60FFBF
:104DB00077980895FF920F931F93CF93DF93EC01A1
:104DC000F42E8C01060F111DF80160816F70B8DFA1
:104DD000F8016081629561704F2DCE01DF91CF9116
:104DE0001F910F91FF90CACF0F931F93CF93DF9323
:104DF0008C01FC0114821582C0E0D0E0F801EC0FB8
:104E0000FD1F80818F7E80834C2F6C2FC801D2DFE5
:104E10002196C430D10591F7DF91CF911F910F9169
:104E20000895E2CFFF920F931F93CF93DF93EC018E
:104E3000888585FF18C08770F82E00E010E04F2DA0
:104E4000400F8F81481778F4FE01E40FF11D808137
:104E500084FD06C06885677061506423CE01AADFB7
:104E60000F5F1F4FECCFDF91CF911F910F91FF90FC
:104E70000895FC016787408B8785208990E0DC01DD
:104E8000AA0FBB1FA80FB91FA20FB11DAA0FBB1FEE
:104E9000A25BBE4F4C9111968C9140878187842FE5
:104EA0008F70893051F047708781242F30E090E077
:104EB0002817390714F4842F01C087818683089549
:104EC000FC018091231C64858B30B1F4662321F0B2
:104ED0001092111C1092101C70E041E050E087818C
:104EE0007817B0F4DF01A70FB11D8C9184FF02C0C9
:104EF000611156C07F5FF3CF662321F010920B1C27
:104F000010920A1C70E041E050E08781781730F081
:104F10008091231C813109F07FC00AC0DF01A70FF7
:104F2000B11D8C9184FF02C061114EC07F5FEDCF37
:104F3000662351F087E090E090930B1C80930A1C4D
:104F40001092111C1092101C70E021E030E087815B
:104F5000781728F5DF01A70FB11D8C9184FF1DC0C4
:104F60008C918F7090E003971CF0611141C015C0C7
:104F7000662399F08C918F704091101C5091111CF8
:104F8000D90102C0AA0FBB1F8A95E2F7CD01842B7D
:104F9000952B9093111C8093101C7F5FD8CF0895A0
:104FA0008C918F702091101C3091111CDA0102C07D
:104FB000AA0FBB1F8A95E2F7CD01822B932B90930A
:104FC000111C8093101C96CF8C918F7020910A1C1D
:104FD00030910B1CDA0102C0AA0FBB1F8A95E2F7C1
:104FE000CD01822B932B90930B1C80930A1C9ECF98
:104FF0008C918F7040910A1C50910B1CD90102C0FA
:10500000AA0FBB1F8A95E2F7CD01842B952B9093B5
:105010000B1C80930A1CC1CF0895EF92FF920F934F
:105020001F93CF93DF93EC01F62E888599859B879C
:105030008A878091231C893031F48A85982F977054
:10504000943009F410C18B856A8580FD11C02D81D3
:1050500030E04F81862F877090E050E084179507ED
:1050600014F08F8190E02817390708F0FAC01C82ED
:1050700066FF22C08D859E8524D98F709881907F90
:10508000982B98838D859E850CD98F709981907F00
:10509000982B998388818061888389818061898345
:1050A00040E060E0CE0186DE41E061E0CE0182DEDC
:1050B000CE01B8DE82E0D0C02E818C8130E090E05D
:1050C000821793070CF01C829D818E81981710F433
:1050D00040E031C0E12C8E81E81680F58C81FE0124
:1050E000E80FF11D00810F7010E06A8567708F81F5
:1050F000262F30E090E0281739070CF06F818D855E
:105100009E85C7D890E00817190759F08C818F5FEA
:105110008C832E818C8130E090E0821793070CF015
:105120001C82E394D8CF8C81FE01E80FF11D8081B1
:1051300084FD08C04F5F8E814817A8F38A8584FDDF
:105140000DC012C08C818F5F8C832E818C8130E0EA
:1051500090E08217930774F31C82ECCF90E02F2D20
:1051600030E04E81941750F087702F8190E030E04E
:10517000821793077CF08F8190E00CC0FE01E90F4D
:10518000F11D40814F7050E04217530709F49C8392
:105190009F5FE7CF2E8130E08217930721F48B8544
:1051A00081FD14C019C010E08E811817C0F78C81E2
:1051B000181751F0FE01E10FF11D80818F7E808371
:1051C000412F60E0CE01DADD1F5FEECFFC828C81E3
:1051D000843010F083E08C838C819F2D9F70FE01C2
:1051E000E80FF11D8081807F892B80838C81FE01F7
:1051F000E80FF11D8081806180834C816C81CE013C
:10520000D9DDCE010FDE6A8563FF0BC08C818F5F15
:105210008C832E818C8130E090E0821793070CF014
:105220001C824D814F5F4D8350E06770862F90E068
:105230002F8130E08217930714F49C0102C02F8164
:1052400030E02417350748F42F8130E082179307A8
:1052500014F4862F01C08F818D83CE0131DE81E071
:1052600009C080E007C09B8591609B878860806152
:105270008A87E9CEDF91CF911F910F91FF90EF9038
:105280000895FF920F931F93CF93DF93EC018885CE
:1052900087FD04C0F12C062F10E02BC08D859E8564
:1052A0000E944321811102C010E009C060E08D8599
:1052B0009E850E944921682FCE01AFDE45C08F81B7
:1052C000181708F040C0FE01E10FF11D80818F7EAC
:1052D0008083412F60E0CE0151DD1F5FF0CFFE01E2
:1052E000EF0DF11D80818F7090E08017910729F0FC
:1052F000F3948F81F81698F310C080818F7E80839D
:105300004F2D60E0CE013ADD8D81882319F08D812B
:1053100081508D83CE0186DDEBCF8D859E850E94E9
:105320004321811111C010E08F81181760F4FE0134
:10533000E10FF11D80818F7E8083412F60E0CE01DF
:105340001DDD1F5FF1CF1D82CE01DF91CF911F9137
:105350000F91FF90B5CDDF92EF92FF920F931F93C5
:10536000CF93DF938C01FC01858596850E944E21A9
:10537000C0E0D0E0F82FFF70DF2EE82EF12CF8010E
:10538000EC0FFD1F8081807F8D29808380818F7E3F
:1053900080834C2F6C2FC801D3DCC7010C2E02C0B8
:1053A000959587950A94E2F780FF03C04C2F61E042
:1053B00002C04C2F60E0C801E1DC2196C430D10569
:1053C000F1F6C801DF91CF911F910F91FF90EF90FF
:1053D000DF9076CDFC01808587702781482F50E0D3
:1053E00030E0421753070CF08781089523E0FC0159
:1053F0002783089524E0FC0127830895FC01878515
:1054000090899370990F990F8370892BE4E2FCE1E6
:1054100090819295917090FB84F99081907E892B78
:10542000089521E0FC0124870895FC011486089565
:10543000CF93DF9300D000D0CDB7DEB79B01AC0196
:10544000611571058105910559F069833A834B8394
:105450005C83C2D429813A814B815C8112D403C020
:1054600060E070E0CB010F900F900F900F90DF91F4
:10547000CF910895CF92DF92EF92FF926B017C0162
:1054800062177307840795075CF4CA01B9016C19A8
:105490007D098E099F09CCDF6C0D7D1D8E1D9F1D22
:1054A000FF90EF90DF90CF90089526D00E94811A50
:1054B0000E940B1EFDCF1DBA109268001CBC10BECE
:1054C0001FBA10927A0010926E0010926F00109224
:1054D0007000109271001092C9001092BC0011B8B7
:1054E00014B817B81AB81DB810BA12B815B818B849
:1054F0001BB81EB811BA0895F894E1E6F0E020E870
:105500002083108283E084BD85BDEEE6F0E08081DB
:105510008160808391E09093800082E0809381009D
:105520009093B0008093B10090939000809391008D
:1055300086E880937A0020937B0010927E006DD0E5
:1055400078940895F89484B7877F84BF8091600031
:105550008061809360001092600080E29EE4019779
:10556000F1F781E08093E00080E28093D80080E64C
:105570009AEE0197F1F79FDF0C9400FEFFCFF894AD
:105580009ADF80E69AEE0197F1F70C940000FFCFC6
:105590008F938FB78F938091041D8D5F8D37D0F4DB
:1055A0008093041D8091051D8F5F8093051DD8F0A9
:1055B0008091061D8F4F8093061DA8F08091071DD6
:1055C0008F4F8093071D78F08091081D8F4F809337
:1055D000081D09C08D578093041D8091051D8E5FA5
:1055E0008093051D28F78091091D8C5F8093091D0C
:1055F00058F080910A1D8F4F80930A1D28F08091EA
:105600000B1D8F4F80930B1D8F918FBF8F9118951E
:105610008091E80080FFFCCF08958091D80087FF3B
:1056200002C085FF1BC081E88093D70080EA809389
:10563000D80086E189BD09B400FEFDCF80E98093E2
:10564000D8001092E0001092111D1092101D1092BF
:105650000F1D1092E1008DE08093E20008951F92EB
:105660000F920FB60F9211240BB60F922F933F9308
:105670004F935F936F937F938F939F93AF93BF935A
:10568000EF93FF938091E1001092E10083FF11C03E
:105690001092E90091E09093EB001092EC0092E2FE
:1056A0009093ED0098E09093F0001092111D1092ED
:1056B0000F1D82FF1DC09091111D9923C9F090917B
:1056C0000E1D992359F0915090930E1D911106C013
:1056D00094E09093E9009AE39093E80090910D1D77
:1056E000992331F0915090930D1D911101C02ADF43
:1056F00080FF0CC090E19093E2001092111D91E0A8
:105700009093101D90EA9093D80019BC9091101DB1
:10571000992379F084FF0DC086E189BD09B400FEAC
:10572000FDCF80E98093D8008DE08093E200109255
:10573000101DFF91EF91BF91AF919F918F917F913C
:105740006F915F914F913F912F910F900BBE0F90F2
:105750000FBE0F901F9018951F920F920FB60F92C9
:1057600011240BB60F92EF92FF920F931F932F937A
:105770003F934F935F936F937F938F939F93AF93D9
:10578000BF93EF93FF93CF93DF931F92CDB7DEB715
:105790001092E9008091E80083FF39C13091F10057
:1057A0002091F100E090F100F090F1000091F10003
:1057B0001091F1008091F1009091F10042EF40933F
:1057C000E800263009F03FC046E0E6EBF0E0259126
:1057D00035912E153F0511F0359615C0259135915F
:1057E0002017310711F033960EC025913591449161
:1057F0008F3F910519F010F08FEF90E0841708F4B7
:10580000482F5EEF08C0415011F701C1481B50936B
:10581000E8004423A9F08091E800982F9570D9F30F
:1058200082FDF8C0842F413208F080E2982F99233E
:1058300069F3F90125912093F1009F019150F7CF71
:10584000803249F3E7C0253049F48EEF8093E800B9
:10585000DFDE8E2D80688093E300DCC0293001F507
:105860003111B2C0E092111D10920F1D10920E1D49
:105870008EEF8093E80081E0E9E7F1E08093E900B2
:1058800095919093EB00992331F095919093EC00D2
:1058900095919093ED008F5F853081F78EE1B2C0D6
:1058A000283049F4303809F08FC0B2DE8091111DE4
:1058B0008093F10085C0213291F4313A09F084C01F
:1058C000A7DEE4E0F1E0CF01019620812093F10012
:1058D00021E08B30920709F473C0FC01F4CF203231
:1058E00009F04AC0313209F06FC08091E80082FFB0
:1058F000FCCFE4E0F1E0CF0101962091F10020839C
:10590000E1E08B309E0711F0FC01F5CF8BEF809327
:10591000E8008EEF8093E80030910401409105018A
:10592000809106012091070190E0A0E0B0E0DC0149
:1059300099278827942B832BB22B86389105A105B4
:10594000B10521F48FE080930D1D64C08639910567
:10595000A105B10509F05EC084E08093E9009FEFE6
:105960008091EE00837039F09093E8008091E80018
:1059700082FDFCCFF5CF03DE223229F4313221F54E
:10598000E0920F1D05C0233229F4313209F03FC0E7
:105990003FDE16C0211118C039833ADE3981323812
:1059A00051F40093E9008091EB0085FB882780F992
:1059B0001092E90001C080E08093F1001092F100A4
:1059C0008EEF8093E80026C0822F8D7F8130F9F41E
:1059D0003230E9F4EF28D9F40F778FEF800F86305B
:1059E000B0F48EEF8093E8000093E900233079F063
:1059F00089E18093EB0081E090E0002E01C0880FE8
:105A00000A94EAF78093EA001092EA0003C081E268
:105A10008093EB000F90DF91CF91FF91EF91BF91B9
:105A2000AF919F918F917F916F915F914F913F9136
:105A30002F911F910F91FF90EF900F900BBE0F9041
:105A40000FBE0F901F90189570D088F09F5790F060
:105A5000B92F9927B751A0F0D1F0660F771F881F93
:105A6000991F1AF0BA95C9F712C0B13081F077D0FA
:105A7000B1E0089574C0672F782F8827B85F39F098
:105A8000B93FCCF3869577956795B395D9F73EF4F2
:105A900090958095709561957F4F8F4F9F4F08959A
:105AA000E89409C097FB3EF49095809570956195B8
:105AB0007F4F8F4F9F4F9923A9F0F92F96E9BB276E
:105AC0009395F695879577956795B795F111F8CFEA
:105AD000FAF4BB0F11F460FF1BC06F5F7F4F8F4F55
:105AE0009F4F16C0882311F096E911C0772321F04B
:105AF0009EE8872F762F05C0662371F096E8862FE3
:105B000070E060E02AF09A95660F771F881FDAF739
:105B1000880F9695879597F9089557FD9058440FEB
:105B2000551F59F05F3F71F04795880F97FB991FFC
:105B300061F09F3F79F087950895121613061406B9
:105B4000551FF2CF4695F1DF08C016161706180646
:105B5000991FF1CF86957105610508940895E89421
:105B6000BB2766277727CB0197F908950BD078C01C
:105B700069D028F06ED018F0952309F05AC05FC0A4
:105B80001124EECFCADFA0F3959FD1F3950F50E01B
:105B9000551F629FF001729FBB27F00DB11D639FDF
:105BA000AA27F00DB11DAA1F649F6627B00DA11D85
:105BB000661F829F2227B00DA11D621F739FB00D2B
:105BC000A11D621F839FA00D611D221F749F33279B
:105BD000A00D611D231F849F600D211D822F762F34
:105BE0006A2F11249F5750408AF0E1F088234AF031
:105BF000EE0FFF1FBB1F661F771F881F915050407D
:105C0000A9F79E3F510570F014C0AACF5F3FECF397
:105C1000983EDCF3869577956795B795F795E79568
:105C20009F5FC1F7FE2B880F911D9695879597F979
:105C3000089597F99F6780E870E060E008959FEF0E
:105C400080EC089500240A94161617061806090613
:105C5000089500240A9412161306140605060895E2
:105C6000092E0394000C11F4882352F0BB0F40F46A
:105C7000BF2B11F460FF04C06F5F7F4F8F4F9F4FAA
:105C80000895052E97FB16F400940FD057FD05D00C
:105C900028D007FC02D046F408C0509540953095B6
:105CA00021953F4F4F4F5F4F089590958095709588
:105CB00061957F4F8F4F9F4F0895EE0FFF1F059007
:105CC000F491E02D09942FD0A59F900DB49F900DD5
:105CD000A49F800D911D112408950790F691E02D49
:105CE0000994A1E21A2EAA1BBB1BFD010DC0AA1F1D
:105CF000BB1FEE1FFF1FA217B307E407F50720F035
:105D0000A21BB30BE40BF50B661F771F881F991FAF
:105D10001A9469F760957095809590959B01AC01F8
:105D2000BD01CF010895A29FB001B39FC001A39F01
:105D3000700D811D1124911DB29F700D811D1124C4
:105D4000911D08958F929F92AF92BF92CF92DF9252
:105D5000EF92FF92CF93DF93EC01688179818A8182
:105D60009B81611571058105910521F464E279ED4E
:105D70008BE597E02DE133EF41E050E082DF490110
:105D80005A019B01AC01A7EAB1E49DDF6B017C01E4
:105D9000ACEEB4EFA501940143D0C60ED71EE81EA9
:105DA000F91EF7FE06C081E0C81AD108E10880E8B4
:105DB000F80AC882D982EA82FB82C701B6019F77BE
:105DC000DF91CF91FF90EF90DF90CF90BF90AF9099
:105DD0009F908F900895B6CF80E091E0B3CF60930D
:105DE00000017093010180930201909303010895D3
:105DF000F999FECF92BD81BDF89A992780B5089593
:105E0000262FF999FECF1FBA92BD81BD20BD0FB6D6
:105E1000F894FA9AF99A0FBE01960895B7FF53CFF6
:0C5E200052DF821B930B0895F894FFCF13
:105E2C000100000000E1000000000800000040C775
:105E3C00C0EA3FFD44D73F2A67C53FF304B53FD7BF
:105E4C00FEA53FF037983FC2958B3F0000803F8204
:105E5C00DD673F7F01523F10353E3F75462C3FA416
:105E6C00081C3FCE520D3F0000003FA8A8A2040022
:105E7C001C010C01E2013A012A01A1019901000067
:065E8C0004030000000009
:00000001FF
